:1000000086015F308C000D3084008001840A8C0BE7
:1000100005282A281F208400073984060310840C31
:10002000840C840C041A841704128A018207013498
:100030000234043408341034203440348034073916
:100040008A01820730343134323433343434353435
:100050003634373407309120FF30FB2001308C00DC
:1000600004308D000C088E004A200D088E004A20B6
:1000700007308D2037301021FF200130EB20031D89
:100080006C28123002210130D220123009210730B1
:100090009420322800308A000E08FA3E03185B28AC
:1000A000063E54208E005B288207403412345234BE
:1000B0001B345B343F340608FF208030CB202208FD
:1000C000860007308A200608FF200E08C420220878
:1000D00086000430992018291230AF201208FF2022
:1000E0000730CB2022088C001308FF200730CB20DC
:1000F00022088D000C08FF200530E620031D6C2827
:100100000D08FF200530E620031D6C284728073026
:10011000A72087280A20800695280A2084178004B3
:1001200018290A20800495280A20FF3A84178005A0
:100130001829A301A200E020640023082204031967
:100140000800F730FF3E031DA228E2209C288316FA
:100150000739F83881006300FF3081001829A400B6
:100160000221B52024080921182923082204031993
:10017000A20A8030221AA3062219A306A218A306F7
:10018000230DA20DA30D0800A501A4002408A204BC
:100190002508A3041829A501A4002408A205250800
:1001A000A3051829A501A400223084002408800793
:1001B0002508840F00000318013E031C800718293E
:1001C000A309A209A20A0319A30A0800A501A40011
:1001D000F02001391829A501A400F02002391829BE
:1001E00025082302031DF8282408220203190234DB
:1001F000031C04340134FF3A831686001829A30136
:10020000A200182984000008A200840A0008A300A4
:100210001829840022088000840A230880001829F5
:100220000B20A9000005841B2906031900340134A2
:06023000831264000800C7
:084000007F007F007F007F00BC
:02400E00FD3F74
:024010000100AD
:00000001FF
